:10000000831600308500073086008312FD20FD2016
:1000100064305A2013200130C72016210130990086
:100020000C309A00A4298030C7204130E22075307E
:10003000E2207430E2207230E2206F30E2206E3035
:10004000E2206930E2206330E2206130E220A0301B
:10005000E2205630E2204230E2205330E220C0302D
:10006000C7206330E220A030E2205330E2202E305F
:10007000E2204430E2206130E2206E30E22069303C
:10008000E2206530E2206C30E2207330E2206530FF
:10009000E2206E30E22005304E2008009800FF304C
:1000A0005A20FF305A20FF305A20FF305A20980B38
:1000B0004F2808009100F93090000618A4298618EE
:1000C000A4290000900B5D28910B5B28080091008B
:1000D000F930900006190800061C8618A429900B18
:1000E0006A28910B682808009501960197019200F3
:1000F0000A309300AD201208950014089200AD203C
:100100001208960014089200AD20120897001708F4
:10011000B620E2201608B620E2201508B620E2201C
:10012000080095019601970192000A309300AD20D6
:100130001208950014089200AD20120896001408C9
:100140009200AD20120897001708B6201608B620B6
:10015000E2201508B620E22008009401130892025C
:10016000031CB428940AAF28920708008207303491
:10017000313432343334343435343634373438343B
:1001800039344134423443344434453446348D00A8
:100190000F121C21162105141621F0308F051C2189
:1001A0008D0E0D080F398F041C2105101621051422
:1001B000F0308F051C218D0E0D080F398F041C2186
:1001C000051008008D000F161C211621051416219C
:1001D000F0308F051C218D0E0D080F398F041C2166
:1001E000051016210514F0308F051C218D0E0D0809
:1001F0000F398F041C210510080016211621162125
:1002000016212030C72016212830C7201621203083
:10021000C72016212830C72016210E30C7201621EE
:100220000130C72016210430C72008008C30900010
:100230000000900B182908000F1806160F1C061254
:100240008F1886168F1C86120F1906170F1D06139E
:100250008F1986178F1D86130F1A86150F1E86118C
:1002600008000C309A028030C7204130E220443030
:10027000E2205230E2204530E2205330E220533079
:10028000E2204530E2203A30E220A030E220190896
:100290009120C030C7204630E220EF30E2204C30C1
:1002A000E2205330E2204F30E2204D30E22048304F
:1002B000E2204530E2205430E2203A30E220A03003
:1002C000E2201A08742008000311061868296D2915
:1002D000990A0C309A0006186B298618702975291E
:1002E00099030C309A0086187329031D792963300D
:1002F000990064301902031C0800013099000800BD
:10030000061D802903305A20061D802906198629DA
:10031000FA305A20061D8A290330061D80299B01C8
:1003200006199029061D9229061994299A019B0AFB
:10033000013067209A0A061D98291B081902031C20
:0E0340008029031D9429A429642131218029DC
:02400E00F13F80
:00000001FF
